:020000040800F2
:100000000000022085280008412700084327000837
:10001000452700084727000849270008000000007E
:100020000000000000000000000000004B27000856
:100030004D270008000000004F2700085127000846
:10004000D5280008D5280008D5280008D52800089C
:10005000D5280008D5280008D5280008D52800088C
:10006000D5280008D5280008D5280008D52800087C
:10007000D5280008D5280008D5280008D52800086C
:10008000D5280008D5280008D5280008D52800085C
:10009000D5280008D5280008D5280008D52800084C
:1000A000D5280008D5280008D5280008D52800083C
:1000B000D5280008D5280008D5280008D52800082C
:1000C000D5280008D5280008D5280008D52800081C
:1000D000D5280008D5280008D5280008D52800080C
:1000E000D5280008D5280008D5280008D5280008FC
:1000F000D5280008D5280008D5280008D5280008EC
:10010000D5280008D5280008D5280008D5280008DB
:10011000D5280008D5280008D5280008D5280008CB
:10012000D5280008D5280008D5280008D5280008BB
:10013000D5280008D5280008D5280008D5280008AB
:10014000D5280008D5280008D5280008D52800089B
:10015000D5280008D5280008D5280008D52800088B
:10016000D5280008D5280008D5280008D52800087B
:10017000D5280008D5280008D52800080000000070
:08018000D5280008D52800086D
:1001900010B5054C237833B9044B13B10448AFF3C1
:1001A00000800123237010BD7400002000000000B7
:1001B0001832000808B5034B1BB103490348AFF3DD
:1001C000008008BD00000000780000201832000800
:1001D000034613F8012B002AFBD1181A0138704787
:1001E00001F0FF01102A2BDB10F0070F08D010F8E8
:1001F000013B013A8B422DD010F0070F42B3F6D1EC
:10020000F0B441EA012141EA014122F007047FF004
:1002100000070023F0E80256083C85EA010586EA5B
:10022000010685FA47F5A3FA87F586FA47F6A5FA97
:1002300087F68EB9EED1F0BC01F0FF0102F00702A3
:1002400032B110F8013B013A83EA010313B1F8D14E
:100250000020704701387047002D06BF354603382F
:10026000073815F0010F07D1013015F4807F02BF68
:10027000013015F4C03F0130F0BC0138704700BFB9
:1002800053B94AB9002908BF00281CBF4FF0FF31FD
:100290004FF0FF3000F088B9ADF1080C6DE904CEE5
:1002A00000F006F8DDF804E0DDE9022304B0704751
:1002B0002DE9F047089D8E4604468846002B4AD11A
:1002C0008A42174662D9B2FA82F64EB1C6F12003CD
:1002D00001FA06F820FA03F3B74043EA0808B440ED
:1002E0004FEA174E1FFA87FCB8FBFEF1230C0EFBFA
:1002F000118843EA084301FB0CF29A4209D9FB1822
:1003000001F1FF3080F0EA809A4240F2E780023942
:100310003B449A1AA3B2B2FBFEF00EFB102243EA52
:10032000024300FB0CFC9C4509D9FB1800F1FF328D
:1003300080F0D6809C4540F2D3803B44023840EAAE
:100340000140A3EB0C0300211DB1F3400022C5E9DD
:100350000032BDE8F0878B4205D90DB1C5E9000137
:1003600000210846F5E7B3FA83F1002946D1734529
:1003700002D3824200F20581841A6EEB030201204F
:100380009046002DE5D0C5E90048E2E7002A00F0DC
:100390009080B2FA82F6002E40F0A4808A1A030CF4
:1003A0004FEA174E80B2BCB20121B2FBFEFC0EFB3D
:1003B0001C2243EA024304FB0CF29A4207D9FB18C1
:1003C0000CF1FF3802D29A4200F2E080C4469B1A38
:1003D000B3FBFEF20EFB123340EA034302FB04F4CC
:1003E0009C4207D9FB1802F1FF3002D29C4200F276
:1003F000CA8002461B1B42EA0C40A5E7C1F1200659
:100400008B4022FA06F71F430EFA01F420FA06F396
:100410002EFA06FE4FEA1749234300FA01F81FFAA5
:1004200087FCBEFBF9F01C0C09FB10EE44EA0E44FD
:1004300000FB0CFEA64502FA01F209D93C1900F1B5
:10044000FF3A80F09C80A64540F2998002383C44F7
:10045000A4EB0E041FFA83FEB4FBF9F309FB13446B
:100460004EEA044403FB0CFCA44508D93C1903F1F3
:10047000FF3E80F08280A4457FD9023B3C4443EAA2
:100480000040A4EB0C04A0FB02EC64457346E1467B
:1004900062D35FD05DB1B8EB030264EB090404FAE8
:1004A00006F622FA01F31E43CC40C5E900640021A0
:1004B0004FE7B1FBF2FC010C41EA0E4180B240EA89
:1004C00001423B4638463C46B846BE462026B1FB74
:1004D000F7F1A2EB080241EA0C4166E7014618E792
:1004E00010462CE7C6F120022EFA02F3B740B140C5
:1004F00020FA02F24FEA174E0A43B3FBFEF8BCB2F1
:100500000EFB1833110C41EA034108FB04F9B0401B
:1005100089454FEA104380B23ED9791808F1FF3C73
:1005200001D289451FD8A1EB0901B1FBFEF909FBF6
:1005300004F80EFB191192B242EA0142424529D257
:10054000BA1809F1FF31C4D24245C2D2A9F1020161
:100550003A44BEE7F0459DD2BEEB02036CEB070CBC
:100560000138E14696E7A7EB09094944A8F1020CD6
:10057000B1FBFEF909FB04F8DBE773467FE7504661
:1005800066E70846FDE63B44023A33E7ACF1020C6D
:100590003B441CE749469CE7A1EB0901C446B1FB7B
:1005A000FEF909FB04F8C4E7704700BF10B5044624
:1005B0000E4B1A784FF47A73B3FBF2F30C4A1068BF
:1005C000B0FBF3F000F0ACF868B90F2C01D90120B2
:1005D0000AE0002221464FF0FF3000F091F8034B73
:1005E0005C60002000E0012010BD00BF0000002082
:1005F0002000002008B50B4B1A6842F400721A6004
:100600001A6842F480621A601A6842F480721A60B2
:10061000032000F063F80020FFF7C8FF02F074F831
:10062000002008BD003C0240034A1168034B1B78C0
:100630000B441360704700BF9000002000000020B2
:10064000014B1868704700BF9000002038B5044681
:10065000FFF7F6FF0546B4F1FF3F02D0044B1B78CD
:100660001C44FFF7EDFF401BA042FAD338BD00BF8A
:1006700000000020002808DB0901C9B200F1604039
:1006800000F5614080F80013704700F00F00090189
:10069000C9B2014B1954704714ED00E000B500F0E9
:1006A0000700C0F1070CBCF1040F28BF4FF0040C89
:1006B000031D062B0FD9C31E4FF0FF3E0EFA0CF0A0
:1006C00021EA000199400EFA03FE22EA0E0241EAF5
:1006D00002005DF804FB0023EEE70000074AD36840
:1006E00023F4E0631B041B0C000200F4E0600343EE
:1006F00043F0BF6343F40033D360704700ED00E084
:1007000010B50446054BD868C0F30220FFF7C6FFBA
:1007100001462046FFF7AEFF10BD00BF00ED00E030
:100720000138B0F1807F0BD24FF0E0235861054AC9
:10073000F02182F823100020986107221A61704787
:100740000120704700ED00E000230F2B00F2DA805B
:10075000F0B583B03AE0072200E00022AA4032431D
:100760000234694D45F82420684A14686FEA0C0287
:1007700024EA0C054E6816F4803F01D04CEA0405CB
:10078000624C2560646802EA04054E6816F4003F76
:1007900001D04CEA04055D4C6560A46802EA0405DA
:1007A0004E6816F4801F01D04CEA0405574CA56032
:1007B000E46822404D6815F4001F01D04CEA0402A1
:1007C000524CE26001330F2B00F29A8001229A40D2
:1007D0000C6804EA020C32EA0404F3D14C68651E8A
:1007E000012D03D9112C01D0122C12D185685E0085
:1007F0000324B44025EA0405CC68B4402C4384604B
:10080000446824EA02044A68C2F300129A40224370
:100810004260C5684FEA430E032202FA0EF2D44347
:1008200025EA02058A6802FA0EF22A43C2604A6883
:10083000022A01D0122A0FD1DD08083550F82570A0
:1008400003F00706B6000F22B24027EA02070A6942
:10085000B2403A4340F82520026814404A6802F04A
:10086000030202FA0EF2224302604A6812F0805F2D
:10087000A8D000220192264A546C44F48044546467
:10088000526C02F480420192019A9C08A51C1E4AF7
:1008900052F8256003F00305AD000F22AA4026EAB6
:1008A00002061C4A90423FF458AF02F58062904223
:1008B0001AD002F58062904218D002F58062904210
:1008C00016D002F58062904214D002F58062904208
:1008D00012D002F58062904210D002F58062904200
:1008E0003FF439AF082239E7012237E7022235E722
:1008F000032233E7042231E705222FE706222DE702
:1009000003B0F0BD704700BF00380140003C01401B
:10091000003802400000024003685A6912F4806FF8
:1009200001D1002070476FF480625A610023036395
:10093000202280F83D2080F83E30026C42F0040214
:10094000026480F83C30012070472DE9F0410746F1
:100950000D4690461E4624E0FFF772FE069BC01A25
:10096000B04200D8EEB900233B63202287F83D2037
:1009700087F83E303A6C42F020023A6487F83C3007
:1009800001201EE03B689C6925EA040C1FFA8CFCE0
:10099000BCFA8CFC4FEA5C1CE04511D1B6F1FF3F7C
:1009A000DAD1C5F30743012BECD13B685B6925EA3B
:1009B000030C1FFA8CFCBCFA8CFC4FEA5C1CEBE7C6
:1009C0000020BDE8F0812DE9F04105460E461746AE
:1009D00098463DE01A6842F400721A602B686FF482
:1009E00080625A6100232B63202285F83D2085F820
:1009F0003E302A6C42F004022A6485F83C30012023
:100A000034E0FFF71DFEA0EB0800B84200D8FFB9A4
:100A100000232B63202285F83D2085F83E302A6C88
:100A200042F020022A6485F83C3001201EE02B6849
:100A30009C6926EA0404A4B2003C18BF0124A4B1B6
:100A40002B685A6912F4806FC4D1B7F1FF3FD8D137
:100A5000C6F30743012BEAD12B685C6926EA04043C
:100A6000A4B2003C18BF0124E9E70020BDE8F081F2
:100A700070B504460D46164623685B6913F0800F77
:100A80001CD12046FFF748FFD0B9B5F1FF3FF3D0A6
:100A9000FFF7D6FD801BA84201D8002DECD1002322
:100AA0002363202284F83D2084F83E30226C42F0FB
:100AB0002002226484F83C30012000E0002070BD58
:100AC0000120FCE72DE9F04385B004460D46914630
:100AD0001F46DDF830800D9E0368196841F480716F
:100AE00019600096434600224FF00111FFF72DFFD9
:100AF00060B9236805F0FE051D613346424626496C
:100B00002046FFF760FF68B1012008E023681B68FA
:100B100013F4807F02D04FF400732364032005B0E8
:100B2000BDE8F0830023039323685A6903929B690D
:100B30000393039B324641462046FFF799FF30B9A5
:100B4000012F0FD123685FFA89F61E61E7E7236C56
:100B5000042B01D00120E2E72268136843F40073FC
:100B60001360F7E723684FEA19221A6132464146BB
:100B70002046FFF77DFF20B923685FFA89F61E61E2
:100B8000CDE7236C042B01D00120C8E7226813684D
:100B900043F400731360F7E7020001002DE9F0470A
:100BA00084B004460D46164699460C9FDDF8348005
:100BB0000268136843F4806313600368196841F4A2
:100BC00080711960CDF800803B4600224FF0011182
:100BD000FFF7BBFE70B95FFA85FA236805F0FE05E2
:100BE0001D6143463A4641492046FFF7ECFE68B195
:100BF000012008E023681B6813F4807F02D04FF4C3
:100C000000732364032004B0BDE8F087002303933E
:100C100023685A6903929B690393039B42463946B2
:100C20002046FFF725FF80B9B9F1010F18D12368DD
:100C3000F6B21E61424639462046FFF719FF68B3F7
:100C4000236C042B24D00120DDE7236C042B01D07E
:100C50000120D8E72268136843F400731360F7E7B4
:100C60002368320A1A61424639462046FFF700FFE0
:100C700018B92368F6B21E61DCE7236C042B01D09F
:100C80000120C0E72268136843F400731360F7E79C
:100C90002268136843F400731360D4E72268136872
:100CA00043F480731360CDF800803B4600224FF080
:100CB00001112046FFF749FE68B922684AF0010396
:100CC000136143463A4609492046FFF77CFE002857
:100CD00099D0012097E723681B6813F4807F02D026
:100CE0004FF40073236403208DE700BF020001006E
:100CF00070B504460D46164623685B6913F0040F71
:100D00001CD12046FFF708FED0B9B5F1FF3FF3D064
:100D1000FFF796FC801BA84201D8002DECD10023E0
:100D20002363202284F83D2084F83E30226C42F078
:100D30002002226484F83C30012000E0002070BDD5
:100D40000120FCE770B505460C4616462B6859692C
:100D500011F0400F29D1596911F0100F15D1FFF78B
:100D60006FFC801BA04201D8002CEFD100232B6325
:100D7000202285F83D2085F83E302A6C42F0200282
:100D80002A6485F83C30012070BD6FF010025A6172
:100D900000232B63202285F83D2085F83E302A6C05
:100DA0002A6485F83C300120EEE70020ECE70000E3
:100DB000002800F0CC8070B5044690F83D30002B40
:100DC00077D0242384F83D302268136823F0010390
:100DD00013602268136843F40043136022681368A9
:100DE00023F40043136000F0E5FD62685A4B9A4219
:100DF00064D85A4B98428CBF00230123002B40F04B
:100E0000A8805749A1FB00318B0C25686A6822F045
:100E10003F0242EA91426A6021680A6A22F03F0278
:100E200066684D4DAE424FD8013313430B622168C3
:100E3000CA6922F44F4222F0FF026568464B9D4288
:100E40004CD8431E6D00B3FBF5F3013340F6FC7044
:100E5000034278D0C3F30B031A43CA6121680B68BD
:100E600023F0C003E269206A024313430B60216848
:100E70008B6823F4034323F0FF032269E0680243F5
:100E800013438B602168CB6823F0FF036269A0697C
:100E900002431343CB602268136843F001031360DD
:100EA00000202064202384F83D30206384F83E0035
:100EB00070BD80F83C3000F0A9FF82E7294B9842D2
:100EC0008CBF0023012399E74FF4967505FB03F3CC
:100ED000254DA5FB03539B090133A6E7A668BEB9C0
:100EE000431E05EB450CB3FBFCF30133C3F30B03CB
:100EF000B3FA83F35B0943BBC6B9431E05EB450553
:100F0000B3FBF5F30133C3F30B0343F40043A3E74F
:100F1000431E05EB850C0CEB8C0CB3FBFCF301338F
:100F2000C3F30B03B3FA83F35B09E4E7431E05EB5A
:100F3000850505EB8505B3FBF5F30133C3F30B031F
:100F400043F4404388E7042386E7012384E7012034
:100F500070470120ACE700BFA08601007F841E001F
:100F600083DE1B43FF083D00D34D62102DE9F043A3
:100F700083B004460F46904699460C9EFFF760FBEF
:100F8000054694F83D00C0B2202803D0022003B0EB
:100F9000BDE8F0830095192301224B492046FFF755
:100FA000D4FC002840F0898094F83C30012B00F0FC
:100FB0008680012384F83C3023681A6812F0010F00
:100FC00003D11A6842F001021A602268136823F400
:100FD00000631360212384F83D30402384F83E30C1
:100FE000002323640A9B6362BDF82C306385638D04
:100FF0002385364BE362019500964B4642463946BF
:101000002046FFF75FFD00285BD1238D002B35D0F4
:101010002A4631462046FFF72BFD20BB626A236833
:1010200012781A61626A531C6362218D013989B298
:101030002185638D9BB2013B9BB263852368586910
:1010400010F0040FE1D00029DFD052781A61636AF2
:1010500001336362238D013B2385638D9BB2013B8A
:101060009BB26385D1E7236C042B01D001208EE76E
:101070002268136843F400731360F7E72A46314689
:101080002046FFF735FE50B1236C042B01D0012020
:101090007DE72268136843F400731360F7E7226862
:1010A000136843F400731360202384F83D30002359
:1010B00084F83E3084F83C3069E7022067E702207C
:1010C00065E7012063E700BF020010000000FFFF9A
:1010D0002DE9F04387B004460F4690469946109E8E
:1010E000FFF7AEFA054694F83D00C0B2202804D0C0
:1010F0000227384607B0BDE8F08300951923012286
:1011000088492046FFF721FC002840F0438194F8ED
:101110003C30012B00F04081012384F83C302368EF
:101120001A6812F0010F03D11A6842F001021A6026
:101130002268136823F400631360222384F83D308F
:10114000402384F83E30002323640E9B6362BDF885
:101150003C306385638D2385734BE3620195009674
:101160004B46424639462046FFF718FD0746002801
:1011700040F01481238D5BB9029323685A6902926F
:101180009A690292029A1A6842F400721A6075E033
:10119000012B0AD0022B1AD00023059323685A6929
:1011A00005929B690593059B68E02268136823F408
:1011B000806313600023039323685A6903929A693A
:1011C0000392039A1A6842F400721A6056E0226889
:1011D000136823F4806313602268136843F4006388
:1011E00013600023049323685A6904929B69049353
:1011F000049B43E02A4631462046FFF7A3FD002822
:1012000040F0CE8023681A69636A1A70636A0133FA
:101210006362238D013B2385638D9BB2013B9BB2AF
:1012200063852BE000953346002240492046FFF7B6
:101230008CFB002840F0B6802268136843F40073EA
:10124000136023681A69636A1A70626A531C6362C6
:10125000238D013B2385638D9BB2013B9BB263854C
:1012600023681B695370636A01336362238D013BFA
:101270002385638D9BB2013B9BB26385238D002B3D
:101280007FD0032B54D8012BB4D0022BCAD00095A9
:101290003346002225492046FFF757FB002840F03F
:1012A00083802268136823F48063136023681A69BB
:1012B000636A1A70636A01336362238D013B23857D
:1012C000638D9BB2013B9BB2638500953346002240
:1012D00016492046FFF739FB002867D122681368BA
:1012E00043F40073136023681A69636A1A70626AB0
:1012F000531C6362238D013B2385638D9BB2013BAD
:101300009BB2638523681B695370636A0133636210
:10131000238D013B2385638D9BB2013B9BB263858B
:10132000ACE700BF020010000000FFFF0400010056
:101330002A4631462046FFF705FD002838D12368AC
:101340001A69636A1A70626A531C6362238D013BD7
:101350002385638D9BB2013B9BB2638523685969EA
:1013600011F0040F8AD01B695370636A0133636202
:10137000238D013B2385638D9BB2013B9BB263852B
:101380007CE7202384F83D30002384F83E3084F845
:101390003C30AEE60227ACE60227AAE60127A8E623
:1013A0000127A6E60127A4E60127A2E60127A0E679
:1013B00001279EE6002800F0DA8170B582B004466D
:1013C000036813F0010F3BD09F4B9B6803F00C03A5
:1013D000042B2CD09C4B9B6803F00C03082B21D0D2
:1013E0006368B3F5803F4FD0B3F5A02F52D0964B32
:1013F0001A6822F480321A601A6822F480221A6075
:101400006368002B50D0FFF71BF905468E4B1B6815
:1014100013F4003F14D1FFF713F9401B6428F5D9EA
:101420000320ABE1884B5B6813F4800FD8D0864B68
:101430001B6813F4003F03D06368002B00F0998110
:10144000236813F0020F54D07F4B9B6813F00C0FEE
:101450003ED07D4B9B6803F00C03082B33D0E36830
:10146000002B68D0794B01221A60FFF7E9F8054696
:10147000754B1B6813F0020F54D1FFF7E1F8401BC6
:101480000228F5D9032079E16F4A136843F48033C9
:101490001360B5E76C4B1A6842F480221A601A6830
:1014A00042F480321A60ABE7FFF7CAF80546664B94
:1014B0001B6813F4003FC3D0FFF7C2F8401B642839
:1014C000F5D903205AE1604B5B6813F4800FC6D155
:1014D0005D4B1B6813F0020F03D0E368012B40F053
:1014E0004A81594A136823F0F803216943EAC1038A
:1014F0001360236813F0080F42D063696BB3534B3A
:101500000122C3F8802EFFF79BF805464E4B5B6F18
:1015100013F0020F34D1FFF793F8401B0228F5D9DE
:1015200003202BE1484A136823F0F803216943EABA
:10153000C1031360DDE7454B00221A60FFF780F816
:101540000546414B1B6813F0020FD2D0FFF778F825
:10155000401B0228F5D9032010E13C4B0022C3F8C0
:10156000802EFFF76DF80546374B5B6F13F0020FC7
:1015700006D0FFF765F8401B0228F5D90320FDE0EF
:10158000236813F0040F77D02F4B1B6C13F0805F90
:1015900033D1002301932C4B1A6C42F080521A6411
:1015A0001B6C03F080530193019B0125284B1B68A2
:1015B00013F4807F23D0A368012B34D0052B38D0BF
:1015C000214B1A6F22F001021A671A6F22F00402EF
:1015D0001A67A368002B3DD0FFF732F806461A4B76
:1015E0001B6F13F0020F46D1FFF72AF8801B41F260
:1015F00088339842F3D90320C0E00025D6E7144A87
:10160000136843F480731360FFF71AF80646104B13
:101610001B6813F4807FCED1FFF712F8801B0228DD
:10162000F5D90320AAE0084A136F43F001031367BA
:10163000CFE7054B1A6F42F004021A671A6F42F0A7
:1016400001021A67C5E700BF0038024000004742A8
:1016500000700040FEF7F4FF06464F4B1B6F13F07F
:10166000020F08D0FEF7ECFF801B41F2883398424E
:10167000F3D9032082E0E5B9A369002B7DD0464A67
:10168000926802F00C02082A51D0022B17D0434B6B
:1016900000221A66FEF7D4FF04463F4B1B6813F086
:1016A000007F42D0FEF7CCFF001B0228F5D90320B3
:1016B00064E0394A136C23F080531364DCE7374B42
:1016C00000221A66FEF7BCFF0546334B1B6813F079
:1016D000007F06D0FEF7B4FF401B0228F5D9032097
:1016E0004CE0E369226A1343626A43EA8213A26A06
:1016F0005208013A43EA0243E26A43EA0263264A95
:101700005360264B01221A66FEF79AFF0446224BCD
:101710001B6813F0007F06D1FEF792FF001B022822
:10172000F5D903202AE0002028E0002026E0012B44
:1017300026D0194B9B6803F48001E269914221D1C4
:1017400003F03F02216A8A421ED1616A47F6C072E5
:101750001A408A421AD103F44032A16A8A4217D150
:1017600003F07063E26A934214D1002006E0012086
:101770007047012002E0012000E0002002B070BDAF
:101780000120FBE70120F9E70120F7E70120F5E759
:101790000120F3E70120F1E7003802400000474252
:1017A00008B5264B9B6803F00C03042B41D0082B93
:1017B00041D1224B5A6802F03F025B6813F4800F5C
:1017C00012D01E4B5968C1F388111D480023A1FB9C
:1017D0000001FEF755FD194B5B68C3F3014301336C
:1017E0005B00B0FBF3F008BD144B5868C0F38810E1
:1017F0004FEA401CBCEB000C6EEB0E0E4FEA8E1352
:1018000043EA9C634FEA8C11B1EB0C0163EB0E03CE
:10181000DB0043EA5173C90011EB000C43F10003F4
:10182000990200234FEA8C2041EA9C51FEF728FDE3
:10183000D1E70348D7E70348D5E700BF00380240A7
:1018400040787D010024F400002800F09B8070B5F2
:101850000D4604464F4B1B6803F00F038B4208D222
:10186000CBB24C4A1370136803F00F038B4240F065
:101870008B80236813F0020F17D013F0040F04D0ED
:10188000454A936843F4E0539360236813F0080FCC
:1018900004D0414A936843F4604393603E4A93689E
:1018A00023F0F003A1680B439360236813F0010F4A
:1018B00032D06368012B21D09A1E012A25D9364ADD
:1018C000126812F0020F61D033498A6822F00302D5
:1018D00013438B60FEF7B4FE06462F4B9B6803F064
:1018E0000C036268B3EB820F16D0FEF7A9FE801BD3
:1018F00041F288339842F0D9032042E0264A126828
:1019000012F4003FE0D101203BE0234A126812F0BC
:10191000007FD9D1012034E01E4B1B6803F00F0378
:10192000AB4207D9EAB21B4B1A701B6803F00F03D6
:10193000AB422DD1236813F0040F06D0164A9368EA
:1019400023F4E053E1680B439360236813F0080F1E
:1019500007D0114A936823F46043216943EAC10325
:101960009360FFF71DFF0C4B9B68C3F303130B4AF7
:10197000D35CD8400A4B18600A4B1868FEF716FE75
:10198000002070BD012070470120FAE70120F8E730
:101990000120F6E7003C024000380240445A0008AB
:1019A0002000002004000020014B1868704700BF91
:1019B0002000002008B5FFF7F7FF044B9B68C3F336
:1019C0008223034AD35CD84008BD00BF00380240E0
:1019D000545A000808B5FFF7E7FF044B9B68C3F3B0
:1019E0004233034AD35CD84008BD00BF00380240F0
:1019F000545A000810B504460268136923F4405392
:101A0000C1680B431361836802691A4343691A432F
:101A1000C3691A430168CB6823F4164323F00C030F
:101A20001343CB600268536923F4407381690B430D
:101A30005361C369B3F5004F35D00368604A9342E0
:101A400000F0918002F58062934200F08C80FFF7F5
:101A5000B1FF0021031849411B1841F10001C900E1
:101A600041EA5371DB00181863684FEA83024FEABA
:101A7000937341F10001FEF703FC524AA2FB0031CF
:101A80004909642303FB11031B013233A2FB032327
:101A90005B0903F0F00202EB011203F00F0321686F
:101AA00013448B608AE00368454A93422FD002F5C5
:101AB000806293422BD0FFF77DFF0023021843EB97
:101AC0000301121841F10001C90041EA5271D2002C
:101AD000101841F10001626892185B41FEF7D0FBDB
:101AE000384AA2FB00314909642303FB1103DB00E0
:101AF0003233A2FB03235B095A0002F4F87202EBB3
:101B0000011203F00703216813448B6056E0FFF7CE
:101B100061FF0023021843EB0301121841F1000199
:101B2000C90041EA5271D200101841F10001626807
:101B300092185B41FEF7A4FB224AA2FB003149093F
:101B4000642303FB1103DB003233A2FB03235B0995
:101B50005A0002F4F87202EB011203F00703216845
:101B600013448B602AE0FFF735FF00210318494139
:101B70001B1841F10001C90041EA5371DB0018183C
:101B800063684FEA83024FEA937341F10001FEF765
:101B900077FB0C4AA2FB00314909642303FB1103C4
:101BA0001B013233A2FB03235B0903F0F00202EBBB
:101BB000011203F00F03216813448B6010BD00BFB6
:101BC000001001401F85EB512DE9F84305460F46F3
:101BD00016469946DDF820802B681C6837EA040415
:101BE0000CBF01240024B4421FD1B8F1FF3FF3D051
:101BF000B8F1000F05D0FEF723FDA0EB090040452A
:101C0000EAD92A68D36823F4D073D3602A68536969
:101C100023F001035361202385F8393085F83A30E9
:101C2000002385F83830032000E00020BDE8F88369
:101C300058B310B5044690F839300BB3242384F818
:101C400039302268D36823F40053D3602046FFF76D
:101C5000D1FE2268136923F490431361226853690B
:101C600023F02A0353612268D36843F40053D360FE
:101C70000020E063202384F8393084F83A3010BD26
:101C800080F8383000F0C6FDD8E7012070472DE914
:101C9000F04383B01E4690F83930DBB2202B56D18A
:101CA00004460D469046002955D0002A55D090F89C
:101CB0003830012B53D0012380F838304FF0000921
:101CC000C0F83C90212380F83930FEF7B9FC074674
:101CD000A4F82480A4F8268084F8389010E00096B8
:101CE0003B46002280212046FFF76EFF002838D1B6
:101CF0002B882268C3F3080353602369CBB90235EC
:101D0000E38C9BB2BBB1E28C92B2013A92B2E28414
:101D1000A368B3F5805FE2D000963B4600228021A5
:101D20002046FFF751FFF0B915F8012B23685A60E0
:101D3000E6E70135E4E700963B46002240212046D5
:101D4000FFF742FF88B9202384F8393000E00220F1
:101D500003B0BDE8F0830120FAE70120F8E7022094
:101D6000F6E70320F4E70320F2E70320F0E70000A2
:101D700084B000220092154B196B41F08001196369
:101D8000196B01F08001009100990192196B41F0EB
:101D900004011963196B01F0040101910199029288
:101DA000196B41F001011963196B01F001010291F6
:101DB000029903921A6B42F002021A631B6B03F042
:101DC00002030393039B04B0704700BF0038024036
:101DD00008B50B480B4B03600B4B4360002383603B
:101DE000C3604FF48042026143618361C361036257
:101DF000FEF7DEFF00B908BD00F064FAFBE700BFA4
:101E00009400002000540040A086010030B589B045
:101E10000023039304930593069307930268154BDD
:101E20009A4201D009B030BD00250195124C236BB8
:101E300043F002032363236B03F002030193019B2E
:101E40004FF4407303931223049301230593032358
:101E500006930423079303A90848FEF775FC02952F
:101E6000236C43F400132364236C03F400130293E4
:101E7000029BD7E7005400400038024000040240B3
:101E800010B582B000238DF807300DF10702022152
:101E9000E22000F011FC68B900238DF807300DF145
:101EA00007020121E22000F007FC044638B9204671
:101EB00002B010BD0446044800F018FCF7E70348E0
:101EC00000F014FCF3E700BF5C5A0008745A0008E5
:101ED00010B582B00446FFF7D3FF08BB8DF807406A
:101EE0000DF107020321E22000F0E6FBE0B90DF15D
:101EF0000701E22000F0F4FBD0B99DF8073003F0B1
:101F00007000702833D013F0100F16D1A4F1F7022F
:101F1000072A12D8DFE802F0101111111011101069
:101F2000154800F0E3FBD9E7144800F0DFFBDEE7DB
:101F3000134800F0DBFBE0E7042013F0200F0AD188
:101F4000A4F1F702072A06D8DFE802F00405050528
:101F500004050404022013F0400F09D1F73C072CBC
:101F600006D8DFE804F00705050507050707002088
:101F700002B010BD0120FBE7885A00089C5A0008F7
:101F8000B05A0008022805D0032805D0012805D141
:101F90000348704703487047034870470348704739
:101FA000BC5A0008C05A0008C45A0008105B000858
:101FB000022A05D0032A05D0012A05D1084470471A
:101FC000401A704701FB00F070470000044B0022EC
:101FD0001A605A609A601A735A739A73704700BFF6
:101FE000E8000020154B5B7B3BB9144A927B22B181
:101FF000124B01221A735A737047012B02D0022B25
:1020000012D070470D4B1B7B012B05D0022B07D044
:102010000A4B01221A737047084B02221A73704749
:10202000064B03221A737047044B1A689A60002209
:102030005A6001221A735A73E3E700BFE8000020D8
:1020400010B50F4B5B7B5BB1012B0CD0022B09D180
:102050000B4C227D21692068FFF7AAFF206001E078
:10206000FFF7B4FF10BD064C61682161227B227529
:10207000A068FFF79DFF206002236373F2E700BFB3
:10208000E800002010B50446124B5B7B6BB9114B86
:102090009B68114A934207DC03EB830300EB430484
:1020A0000C4B9C6001229A7310BD012B0BD1094B84
:1020B0005B68094A9342F7DC03EB830300EB4303BD
:1020C000044A5360F0E7FFF781FF024B9C60012256
:1020D0009A73E9E7E8000020FFE0F50508B5FE2067
:1020E000FFF7F6FE042821D0022821D0012821D0B4
:1020F000FD20FFF7EDFE04281ED002281ED0012887
:102100001ED0FB20FFF7E4FE04281BD002281BD0C2
:1021100001281BD0F720FFF7DBFE042818D0022887
:1021200019D0012819D06FF0630000E0012008BD2C
:102130000220FCE70320FAE70420F8E70520F6E791
:102140000620F4E70720F2E70820F0E70920EEE791
:102150004FF0FF30EBE70020E9E76FF00100E6E722
:1021600070B5002000F04CF90021502000F08AFAF0
:10217000464C012394E80600454800F06BFA0C2118
:10218000502000F07FFA012394E80600414800F057
:1021900061FA1821502000F075FA012394E8060036
:1021A0003D4800F057FA2421502000F06BFA01233B
:1021B00094E80600394800F04DFA0021084600F086
:1021C00061FA374B5B7BDBB1012B32D0344C54F8D6
:1021D000182B3449204600F07FFB334A012306CAFE
:1021E000204600F037FA1C21002000F04BFA274A65
:1021F000012306CA2D4800F02DFA00F011F970BD38
:10220000274B03F118049A682949204600F064FB23
:10221000254A012306CA204600F01CFA1C21002092
:1022200000F030FA194A012306CA224800F012FAD7
:10223000E3E71B4DAE68287BFFF7A4FE034605F1DC
:10224000180432461C49204600F046FB1B4A012375
:1022500006CA204600F0FEF91421002000F012FA10
:102260006A681349204600F037FB0F4A012306CA6B
:10227000204600F0EFF93021002000F003FA034A75
:10228000012306CA0E4800F0E5F9B6E71800002061
:10229000C85A0008D05A0008D85A0008E05A000866
:1022A000E80000200C5B000808000020145B000818
:1022B000E85A0008EC5A0008F85A000810000020FC
:1022C000005B0008FEE7000000B595B03022002159
:1022D00008A800F023FB00230393049305930693BF
:1022E00007930193214A116C41F080511164126CE3
:1022F00002F080520192019A02931D4B1A6842F437
:1023000080421A601B6803F480430293029B0123FE
:1023100008934FF48033099302230E934FF4800205
:102320000F92192210924FF4A87211921293042363
:10233000139308A8FFF73EF898B90F2303930223DD
:102340000493002305934FF4A05306934FF4805356
:102350000793052103A8FFF777FA20B915B05DF8B8
:1023600004FBFFF7AFFFFFF7ADFF00BF00380240EF
:102370000070004038B5FEF73DF9FFF7A5FFFFF705
:10238000F7FCFFF725FD00F02BFA00F071F8FFF7DE
:10239000E7FE6FF0630507E0FFF774FEFFF7E0FE6E
:1023A0006420FEF753F92546FFF798FE0446854260
:1023B000F6D010F1640FF3D00028EDDAB0F1FF3F52
:1023C00005D010F1020FE9D1FFF73AFEE6E7FFF77B
:1023D00009FEE3E700B587B08DF817000A230293E2
:1023E000012301930DF11702009200227821034886
:1023F000FEF7BCFD07B05DF804FB00BF94000020B1
:10240000002303E0FF21054AD1540133B3F5806F67
:1024100003D20028F6D10146F5E7704720010020DD
:1024200010B584B000241AE0A4F15000C0B2FFF748
:10243000D1FF0020FFF7CEFF1020FFF7CBFF642372
:10244000029380230193084B03EBC41300930123F1
:10245000402278210548FEF789FD0134E4B2072CBB
:10246000E2D904B010BD00BF20010020940000207C
:1024700008B56420FEF7EAF8AE20FFF7ABFF202096
:10248000FFF7A8FF1020FFF7A5FFB020FFF7A2FF7E
:10249000C820FFF79FFF0020FFF79CFF1020FFF7E9
:1024A00099FF4020FFF796FF8120FFF793FFFF2061
:1024B000FFF790FFA120FFF78DFFA620FFF78AFF0F
:1024C000A820FFF787FF3F20FFF784FFA420FFF736
:1024D00081FFD320FFF77EFF0020FFF77BFFD52091
:1024E000FFF778FFF020FFF775FFD920FFF772FFA5
:1024F0002220FFF76FFFDA20FFF76CFF1220FFF7B3
:1025000069FFDB20FFF766FF2020FFF763FF8D20C8
:10251000FFF760FF1420FFF75DFFAF20FFF75AFFC2
:102520000020FFF76DFFFFF77BFF054B0022A3F8AC
:102530000024A3F80224012083F8050408BD00BF8D
:102540002001002010F0800F26D13F2924D810B49C
:10255000124B93F8043413B1B2FA82F25209012AF1
:102560000FD0CB0800EBC3100C4C225C01F007012C
:1025700001238B40DB435BB2134023545DF8044BD3
:102580007047CB0800EBC310044C235C01F007013B
:102590008A4013432354F1E7704700BF2001002015
:1025A0002DE9F04782B0814602A800E9060098466E
:1025B000274BB3F800349DF8006033447F2B42DC96
:1025C000234BB3F802349DF801A053443F2B3CDC6D
:1025D000002523E01E4BB3F80004B3F8021429448D
:1025E0002044B8FA88F25209C9B2C0B2FFF7AAFF74
:1025F0000134A64211D907FA04F313F4004FE9D0CD
:10260000134BB3F80004B3F80214294420444246A3
:10261000C9B2C0B2FFF796FFEAE70135AA4508D96B
:10262000A9F1200303FB0A53019A32F81370002426
:10263000DFE7074AB2F800343344A2F800344846D2
:1026400002B0BDE8F0870020FAE70020F8E700BFFD
:102650002001002030B583B0044602A800E906003E
:102660001D4600E00134207848B12B4602AA12E949
:102670000600FFF795FF024620788242F2D003B0B1
:1026800030BD0000024BA3F80004A3F80214704709
:102690002001002000B585B064230293012301933B
:1026A00000920A4640EA03010248FEF711FD05B018
:1026B0005DF804FB9400002000B585B020F0010017
:1026C000642302930123019300920A4601460348C2
:1026D000FEF74CFC05B05DF804FB00BF9400002041
:1026E00008B50A460021FFF7D5FF08BD10B504461E
:1026F000FDF76EFD4FF47A7382B221460148FFF771
:10270000C6FA10BD3005002082B0002100910B4BAD
:102710005A6C42F480425A645A6C02F4804200922D
:10272000009A01911A6C42F080521A641B6C03F0FB
:1027300080530193019B02B0704700BF00380240F4
:102740007047FEE7FEE7FEE7FEE770477047704719
:1027500008B5FDF769FF08BD08B503460B4A1268C6
:1027600042B10A4A106803446A46934206D8074AAF
:10277000136008BD054A06491160F2E700F0D6F87B
:102780000C2303604FF0FF30F3E700BF2805002063
:10279000B80600200F49D1F8883043F47003C1F81F
:1027A00088300D4B1A6842F001021A6000209860D0
:1027B0001A6822F0847222F480321A60074A5A6042
:1027C0001A6822F480221A60D8604FF000638B6090
:1027D000704700BF00ED00E00038024010300024D8
:1027E00008B50A480A4B03604FF4E1334360002305
:1027F0008360C36003610C2242618361C361FFF7A0
:1028000017FA00B908BDFFF75DFDFBE730050020B2
:102810000014014000B589B000230393049305938D
:10282000069307930268154B9A4202D009B05DF8EF
:1028300004FB0021019103F592335A6C42F020020F
:102840005A645A6C02F020020192019A02911A6BAA
:1028500042F004021A631B6B03F004030293029B11
:10286000C0230393022304930323069308230793AF
:1028700003A90348FDF768FFD8E700BF0014014033
:1028800000080240DFF834D0002103E00C4B5B5815
:10289000435004310B480C4B42189A42F6D30B4A72
:1028A00002E0002342F8043B094B9A42F9D3FFF7B8
:1028B00071FF00F041F8FFF75DFD70470000022056
:1028C000645B0008000000207400002074000020F9
:1028D000B8060020FEE700000EB410B59DB01FAB97
:1028E000029006906FF000410A48079104910A494E
:1028F00053F8042B0591002402A9006801931B944E
:1029000000F094F9029B1C701DB0BDE8104003B0AC
:10291000704700BF240000200802FFFF0244034666
:10292000934200D1704703F8011BF9E7014B186887
:10293000704700BF2400002070B50D4D0D4C641B86
:10294000A4100026A64209D10B4D0C4C00F064FCEB
:10295000641BA4100026A64205D170BD55F8043BA7
:1029600098470136EEE755F8043B98470136F2E701
:102970005C5B00085C5B00085C5B0008605B000857
:102980007047704738B50546002941D051F8043CDE
:102990000C1F002BB8BFE41800F0E0F81D4A1368C4
:1029A00033B9636014602846BDE8384000F0DCB8F5
:1029B000A34208D9206821188B4201BF19685B68BF
:1029C00009182160EDE71A465B680BB1A342FAD9FA
:1029D00011685018A0420BD120680144501883425E
:1029E0001160E0D118685B68536008441060DAE752
:1029F00002D90C232B60D6E7206821188B4204BF34
:102A000019685B68636004BF091821605460CAE7F5
:102A100038BD00BFB406002070B50F4E0C463168BB
:102A2000054611B900F0A4FB30602146284600F0AD
:102A30009FFB431C03D14FF0FF34204670BDC41CE4
:102A400024F00304A042F8D0211A284600F090FB9D
:102A50000130F2D1EFE700BFB00600202DE9F843C6
:102A6000CD1C25F0030508350C2D38BF0C25002D95
:102A7000064601DBA94204D90C2333600020BDE8DF
:102A8000F883DFF8D48000F069F8D8F800301C46ED
:102A900044BB29463046FFF7BFFF431C044658D1CC
:102AA000D8F800402746002F43D1002C4BD0236894
:102AB0003946304604EB030900F05AFB814542D108
:102AC00021686D1A29463046FFF7A6FF01303AD03B
:102AD00023682B442360D8F800305A6862BBC8F8DA
:102AE00000700FE02268521B20D40B2A17D96119FD
:102AF000A342256018BF5960636808BFC8F800107A
:102B000062514B60304600F02FF804F10B00231D9A
:102B100020F00700C21A1CBF1B1AA350AFE762685F
:102B2000A3420CBFC8F800205A60EBE72346646854
:102B3000AEE73C467F68B6E71A465B68A342FBD126
:102B400000235360DEE70C233360304600F00CF8BE
:102B500094E70560D6E700BFB40600200148FFF700
:102B60000FBF00BFAC0600200148FFF70ABF00BF3F
:102B7000AC0600202DE9F0478E681F46BE420B6868
:102B800082460C4690462DD8B1F90C2012F4906F75
:102B900026D06569096905EB4505A3EB010905EB3D
:102BA000D5757B1C4B446D109D4238BF1D465305A7
:102BB00027D52946FFF752FF064660B321694A46EA
:102BC00000F0E6FAA38923F4906343F08003A38125
:102BD000266165614E44A5EB09052660A5603E4669
:102BE000BE4200D93E4620683246414600F0A6FA71
:102BF000A3689B1BA3602368334423600020BDE8C7
:102C0000F0872A4600F0D2FA06460028E0D1216972
:102C10005046FFF7B7FE0C23CAF80030A38943F0F3
:102C20004003A3814FF0FF30E9E700002DE9F04FAA
:102C300098468B891B069DB007460D46144610D555
:102C40000B6973B94021FFF709FF2860286130B98B
:102C50000C233B604FF0FF301DB0BDE8F08F4023E8
:102C60006B610023099320238DF82930CDF80C8067
:102C70003023DFF89C818DF82A304FF0010923467C
:102C80009A4613F8012B0AB1252AF9D1BAEB040BA5
:102C90000BD05B46224629463846FFF76BFF0130D2
:102CA00000F0A780099A5A4409929AF80030002B44
:102CB00000F09F8000234FF0FF32CDE905230AF199
:102CC000010A049307938DF853301A935446052252
:102CD00014F8011B4E48FDF783FA049AD8B9D006C0
:102CE00044BF20238DF85330110744BF2B238DF8A8
:102CF00053309AF800302A2B15D0079A54460020FA
:102D00004FF00A0C214611F8013B303B092B4BD9FF
:102D1000B0B1079214E0A0EB080309FA03F31343E0
:102D20000493A246D2E7039B191D1B680391002B55
:102D3000BBBF5B4242F0020207930793B8BF049205
:102D400023782E2B0AD163782A2B32D1039B1A1DAC
:102D50001B68039243EAE37302340593DFF8C0A0D3
:102D6000217803225046FDF73BFA38B1049BA0EBD3
:102D70000A004022824013430134049314F8011BDB
:102D800024488DF828100622FDF72AFA002836D0AC
:102D9000214B1BBB039B073323F00703083303932B
:102DA000099B334409936AE70CFB02320C4601206D
:102DB000A8E700230134059319464FF00A0C20467A
:102DC00010F8012B303A092A03D9002BC6D00591FF
:102DD000C4E70CFB012104460123F0E703AB009399
:102DE0002A460E4B04A93846AFF30080421C064623
:102DF000D6D1AB895B063FF52DAF09982CE703AB25
:102E000000932A46054B04A9384600F079F8EDE70F
:102E1000205B00082A5B000800000000752B0008FA
:102E2000265B00082DE9F047164698468A680B692C
:102E3000DDF820909342B8BF1346336091F84320E9
:102E400007460C460AB1013333602368990642BF36
:102E5000336802333360256815F0060506D104F1A6
:102E6000190AE36832689B1AAB4226DC94F84330B7
:102E70002268003B18BF012392062BD404F14302C1
:102E800041463846C84701301ED02368226903F006
:102E90000603042B02BFE5683368ED1AA3680CBF74
:102EA00025EAE57500259342C4BF9B1AED1800265C
:102EB0001A34B5421AD1002008E001235246414697
:102EC0003846C847013003D14FF0FF30BDE8F087E6
:102ED0000135C6E7E1185A1C302081F8430022442E
:102EE00094F8451082F843100233C7E701232246C5
:102EF00041463846C8470130E6D00136D9E70000E0
:102F00002DE9FF470F7E0C9E782F914680460C4698
:102F10009A4601F1430207D8622F0AD8002F00F029
:102F2000D180582F00F0B88004F1420684F8427036
:102F30003AE0A7F16303152BF6D801A151F823F06D
:102F4000992F0008AD2F0008292F0008292F00080D
:102F5000292F0008292F0008AD2F0008292F00086D
:102F6000292F0008292F0008292F0008AB3000085E
:102F7000D72F000865300008292F0008292F0008E6
:102F8000CD300008292F0008D72F0008292F00086E
:102F9000292F00086D30000833681A1D1B68326045
:102FA00004F1420684F8423001239CE03368206833
:102FB000191D3160060601D51D6803E04506FBD5E5
:102FC000B3F90050002D03DA2D236D4284F843300D
:102FD00058480A2311E021683368080653F8045B57
:102FE00002D4490648BFADB26F2F5248336014BFB8
:102FF0000A230823002184F843106668A660002E87
:1030000005DB21682E4321F0040121604BD01646D8
:10301000B5FBF3F103FB1157C75D06F8017D2F46A1
:10302000BB420D46F4D9082B0BD12368DF0708D526
:10303000236961689942DEBF302306F8013C06F13E
:10304000FF36921B2261CDF800A04B4603AA214611
:103050004046FFF7E7FE01304AD14FF0FF3004B0A1
:10306000BDE8F087236843F02003236032487827C7
:1030700084F84570236831681F0651F8045B02D458
:103080005F0648BFADB23160D90744BF43F02003AB
:1030900023601DB11023ADE72648E9E7236823F03C
:1030A00020032360F6E71646BDE7336825686169AB
:1030B000181D30602E061B6801D5196002E06806F5
:1030C000FBD51980002323611646BCE733681A1D1F
:1030D00032601E68626800213046FDF781F808B151
:1030E000801B606063682361002384F84330AAE793
:1030F0002369324649464046D0470130ADD0236867
:103100009B0713D4E068039B9842B8BF1846A6E714
:103110000123324649464046D04701309DD0013513
:10312000E36803995B1AAB42F2DCEBE7002504F19C
:103130001906F5E7315B0008425B0008884210B5CC
:1031400001EB020402D98442234607D8431EA14260
:1031500008D011F8012B03F8012FF8E702440146CB
:103160008A4200D110BD13F8014D02F8014DF7E776
:1031700038B5064D0023044608462B60FFF7ECFAED
:10318000431C02D12B6803B1236038BDA806002080
:103190000A44914200F1FF3300D1704710B511F895
:1031A000014B03F8014F9142F9D110BD2DE9F041D7
:1031B000074614460D4621B9BDE8F0411146FFF718
:1031C0004DBC2AB9FFF7DEFB25462846BDE8F08155
:1031D00000F01AF88442064602D8B4EB500FF4D837
:1031E00021463846FFF73AFC804608B94546ECE7E9
:1031F000B4422246294628BF3246FFF7C9FF294676
:103200003846FFF7BFFBF1E751F8043C181F002BCD
:10321000BCBF0B58C0187047F8B500BFF8BC08BC5D
:103220009E467047F8B500BFF8BC08BC9E46704784
:10323000000000000000000000000000000000008E
:10324000000000000000000000000000000000007E
:10325000000000000000000000000000000000006E
:1032600000000000E003E003E003E003E003E0030C
:10327000E003E003C003C003C001C001C001C001FE
:10328000C001000000000000E003E003E0030000D4
:1032900000000000000000003C1E3C1E3C1E3C1EC6
:1032A0003C1E3C1E3C1E0000000000000000000010
:1032B000000000000000000000000000000000000E
:1032C000000000000000000000000000CE01CE035E
:1032D000DE039E039C039C07FF3FFF7F3807380FE8
:1032E000780F780F780EFFFFFFFFF01EF01CE01C38
:1032F000E03CE03DE039000000000000000000007C
:10330000FC03FE0FEE1FE01EE01EE01EE01EE01FAD
:10331000E00FE007F003FC01FE01FE01FE01FE01EB
:10332000FE01FE01FE3DFC3FF00FE001E001000068
:1033300000000000033E07F78FE78EE79EE3BCE343
:10334000B8E7F8E7F0F7E03FC001FF03FF07F30736
:10335000F30FF31EF33CF338F3787FF03FE0000007
:103360000000000000000000E007F80F780F781F51
:10337000781F781F780FF00FE00F801FC37FC3FB0B
:10338000E7F3F7F1F7F0FFF07FF03EF87F7CFF3FC7
:10339000EF1F00000000000000000000E003E00359
:1033A000E003E003E003C003C001000000000000F0
:1033B000000000000000000000000000000000000D
:1033C00000000000000000000000000000000000FD
:1033D0003F007C00F001E001C003C00780078007C8
:1033E000800F000F000F000F000F000F000F800F65
:1033F00080078007C007C003E001F0017C003F00A8
:103400000F000000007E001FC007C003E001F001B4
:10341000F000F000F800780078007800780078007C
:103420007800F800F000F000F001E001C003C007F0
:10343000001F007E00780000E003C003C001CE3909
:10344000FF3F7F3F20037003F807780F3C1F3806CB
:10345000000000000000000000000000000000006C
:10346000000000000000000000000000000000005C
:103470000000000000000000C001C001C001C00148
:10348000C001C001C001FFFFFFFFC001C001C001BA
:10349000C001C001C00100000000000000000000E9
:1034A000000000000000000000000000000000001C
:1034B000000000000000000000000000000000000C
:1034C0000000E003E003E003E003E001E001E001CD
:1034D000C0018003000000000000000000000000A8
:1034E00000000000000000000000FE3FFE3F000062
:1034F00000000000000000000000000000000000CC
:1035000000000000000000000000000000000000BB
:1035100000000000000000000000000000000000AB
:1035200000000000000000000000E003E003E003F2
:10353000E003000000000000000000000F000F008A
:103540001E001E003C003C0078007800F000F000F7
:10355000E001E001C003C00380078007000F000FF7
:10356000001E001E003C003C0078007800F00000C7
:10357000F007F80F7C1F3E3E1E3C1F7C1F7C0F781F
:103580000F780F780F780F780F780F781F7C1F7CDB
:103590001E3C3E3E7C1FF80FF007000000000000BC
:1035A00000000000F000F007F03FF03FF001F001F4
:1035B000F001F001F001F001F001F001F001F00183
:1035C000F001F001F001F001F001FF3FFF3F0000CA
:1035D0000000000000000000E00FF83F7C3C3C00D1
:1035E0003E003E003E003C003C007C00F800F00144
:1035F000E003C0078007000F001E003E003CFE3FB6
:10360000FE3F00000000000000000000F00FF81F67
:103610007C1C3E003E003E003C003C00F800F00FE9
:10362000F80F7C003E001E001E001E001E003E0023
:103630007C1CF81FE01F00000000000000000000DC
:103640007800F800F800F801F803F807F807780F99
:10365000781E781E783C78787878FFFFFFFF780036
:103660007800780078007800780000000000000002
:1036700000000000FC1FFC1FFC1F001E001E001E9F
:10368000001E001EE01FF81FFC007C003E003E00F4
:103690001E003E003E003C007C1CF81FE01F0000A6
:1036A0000000000000000000FC01FE078E0F001F5C
:1036B000001E003E003C003CF83DFC3F3E7F1F7E6C
:1036C0000F3C0F3C0F3C0F3C0F3E1F1E3E1FFC0FDC
:1036D000F00300000000000000000000FF3FFF3F7B
:1036E000FF3F0F001E001E003C0038007800F00075
:1036F000F000E001E001C003C0038007800F800FED
:10370000000F001F001F000000000000000000006C
:10371000F807FC0F3E1F1E1E1E3E1E3E1E1E3C1FB7
:10372000F80FF007F80FFC1E3E3E1F3C1F7C0F7C7D
:103730000F7C1F3C3E3FFC1FF00700000000000014
:1037400000000000F007F80F7C1E3E3C1E3C1F7C72
:103750001F7C1F7C1F7C1F3C3F3EFF1FEF071F008D
:103760001E001E003E003C00F838F03FE01F000045
:103770000000000000000000000000000000000049
:1037800000000000E003E003E003E00300000000AD
:1037900000000000000000000000E003E003E00380
:1037A000E003000000000000000000000000000036
:1037B0000000000000000000E003E003E003E0037D
:1037C0000000000000000000000000000000E00316
:1037D000E003E003E003E001E001E001C003800357
:1037E00000000000000000000000000003000F00C7
:1037F0003F00FC00F003C00F003F00FE003FC00F81
:10380000F003FC003F000F00030000000000000078
:1038100000000000000000000000000000000000A8
:103820000000000000000000FFFFFFFF000000009C
:103830000000FFFFFFFF000000000000000000008C
:103840000000000000000000000000000000000078
:103850000000000000E000F8007E801FE007F80193
:103860007E001F007E00F801E007801F007E00F848
:1038700000E000000000000000000000F01FFC3F1E
:103880003E381F381F381E001E003C007800F00034
:10389000E001C003C003C007C00700000000000033
:1038A000C007C007C00700000000000000000000C3
:1038B000F803FE0F1E1F0F3E7F3CFF78EF79C773A2
:1038C000C7F38FF38FF38FF39FF39FF3FF73FF7BA8
:1038D000F779003C1C1FFC0FF803000000000000FB
:1038E00000000000000000000000E003E003F0071B
:1038F000F007F007780F780F7C0E3C1E3C1E3E3C14
:10390000FE3FFF3F1F780F780FF007F007F0000031
:103910000000000000000000000000000000F83F70
:10392000FC3F3E3C1E3C1E3C1E3C3E3C7C3CF03F73
:10393000F83F7E3C1F3C1F3C0F3C0F3C1F3CFE3FB2
:10394000F83F000000000000000000000000000040
:103950000000FF01FF07871F003E003C007C00784D
:103960000078007800780078007C007C003E003F02
:10397000831FFF07FF01000000000000000000009F
:10398000000000000000F07FFC7F7E781F781F7829
:103990000F780F780F780F780F780F780F780F78EF
:1039A0001F781E787E78F87FE07F0000000000001E
:1039B00000000000000000000000FF3FFF3F003E4D
:1039C000003E003E003E003E003EFE3FFE3F003E09
:1039D000003E003E003E003E003EFF3FFF3F000035
:1039E0000000000000000000000000000000FF1FB9
:1039F000FF1F001E001E001E001E001E001EFF1FD7
:103A0000FF1F001E001E001E001E001E001E001EC6
:103A1000001E000000000000000000000000000088
:103A20000000FE03FF0F871F003E007C007C007833
:103A300000F800F87FF87FF80F780F7C0F7C0F3EBE
:103A40008F1FFF0FFE0300000000000000000000B9
:103A50000000000000001F7C1F7C1F7C1F7C1F7C5F
:103A60001F7C1F7C1F7CFF7FFF7F1F7C1F7C1F7CB8
:103A70001F7C1F7C1F7C1F7C1F7C0000000000003F
:103A800000000000000000000000FF3FFF3FE003D7
:103A9000E003E003E003E003E003E003E003E0030E
:103AA000E003E003E003E003E003FF3FFF3F00002B
:103AB0000000000000000000000000000000FC1FEB
:103AC000FC1F7C007C007C007C007C007C007C0077
:103AD0007C007C007C007C0078007800F838F03FA7
:103AE000C03F0000000000000000000000000000D7
:103AF00000001F3C1E3C3C3C783CF03CE03DE03F7D
:103B0000C03F803FC03FE03FF03DF03C783C7C3C14
:103B10003E3C1F3C0F3C0000000000000000000085
:103B2000000000000000003E003E003E003E003E5F
:103B3000003E003E003E003E003E003E003E003E95
:103B4000003E003E003EFF3FFF3F0000000000003F
:103B5000000000000000000000001FF81FFC1FFC18
:103B60003FFE3FFE3FFE7FFF77FF77FFF7F7E7F768
:103B7000E7F3E7F3C7F307F007F007F007F00000FB
:103B800000000000000000000000000000000F7CAA
:103B90000F7C0F7E0F7F0F7F8F7F8F7FCF7FEF7B1D
:103BA000EF79FF79FF78FF787F783F783F781F784B
:103BB0001F7800000000000000000000000000006E
:103BC0000000F007FC1F3E3E1F7C0F780F780FF8B7
:103BD0000FF80FF80FF80FF80FF80F780F781F7C19
:103BE0003E3EFC1FF0070000000000000000000047
:103BF000000000000000FC3FFF3F1F3E0F3E0F3E55
:103C00000F3E0F3E1F3E3F3EFC3FF03F003E003E5A
:103C1000003E003E003E003E003E0000000000006E
:103C200000000000000000000000F007FC1F3E3E06
:103C30001F7C0F780F780FF80FF80FF80FF80FF8B8
:103C40000FF80F780F781F7C3E3EFC1FF8077C00B2
:103C50003F000F0003000000000000000000F03FE4
:103C6000FC3F7E3C3E3C1E3C1E3C3E3C3C3CFC3C07
:103C7000F03FE03FF03DF83C7C3C3E3C1E3C1F3CAE
:103C80000F3C0000000000000000000000000000E9
:103C90000000FC07FE1F0E3E003C003C003C003EC6
:103CA000C01FF80FFE037F001F000F000F001F2032
:103CB0003E3CFC3FF01F0000000000000000000040
:103CC000000000000000FFFFFFFFE003E003E0034F
:103CD000E003E003E003E003E003E003E003E003CC
:103CE000E003E003E003E003E00300000000000065
:103CF000000000000000000000000F7C0F7C0F7C23
:103D00000F7C0F7C0F7C0F7C0F7C0F7C0F7C0F7C5B
:103D10000F7C0F7C1E3C1E3C3E3EFC1FF00700004B
:103D2000000000000000000000000000000007F09C
:103D300007F007F80F780F7C1E3C1E3C1E3E3C1E11
:103D40003C1F781F780FF80FF007F007F007E0032B
:103D5000E003000000000000000000000000000080
:103D6000000003E003F003F007F0E7F3E7F3E7F305
:103D7000E773F77BF77FFF7F7F7F7F7F7E7F7E3FCD
:103D80003E3E3E3E3E3E00000000000000000000BF
:103D900000000000000007F80F7C1E3E3E3E3C1F66
:103DA000F80FF007E007E003E003F007F80F7C0FDF
:103DB0007C1E3E3C1F780F780FF0000000000000D2
:103DC0000000000000000000000007F807780F7CEA
:103DD0001E3C1E3E3C1F780FF80FF007E003E00387
:103DE000E003E003E003E003E003E003E00300009E
:103DF0000000000000000000000000000000FF7F45
:103E0000FF7F0F001F003E007C00F800F000E00183
:103E1000E003C007800F000F001E003E007CFF7F04
:103E2000FF7F00000000000000000000FF07800787
:103E3000800780078007800780078007800780074A
:103E4000800780078007800780078007800780073A
:103E500080078007800780078007FF07FF070000B3
:103E600000780078003C003C001E001E000F000F90
:103E700080078007C003C003E001E001F000F0000C
:103E8000780078003C003C001E001E000F000F0070
:103E900007000000F07FF000F000F000F000F000FC
:103EA000F000F000F000F000F000F000F000F00092
:103EB000F000F000F000F000F000F000F000F00082
:103EC000F000F07FF07F0000C000C001C001E003FF
:103ED000E003F007F0077807780F380F3C1E3C1E10
:103EE0001E3C1E3C0F380F780778000000000000D1
:103EF00000000000000000000000000000000000C2
:103F000000000000000000000000000000000000B1
:103F100000000000000000000000000000000000A1
:103F2000000000000000FFFFFFFF00000000000095
:103F3000F000000000000000000000000000000091
:103F40000000000000000000000000000000000071
:103F50000000000000000000000000000000000061
:103F60000000000000000000000000000000000051
:103F7000F80FFC3F7C3C3E003E003E00FE07FE1F6B
:103F80003E3E3E7C3E783E7C7E7CFF3FCF1F000065
:103F90000000000000000000003C003C003C003C31
:103FA000003C003CF83DFE3F3E3F1F3E0F3C0F3CB7
:103FB0000F3C0F3C0F3C0F3C1F3C1E3C3E3FFC3F68
:103FC000F03B0000000000000000000000000000C6
:103FD0000000000000000000FE03FF0F871F003EEE
:103FE000003E003C007C007C007C003C003E003E2B
:103FF000871FFF0FFE03000000000000000000000C
:104000001F001F001F001F001F001F00FF07FF1FD2
:104010003F3E1F3C1F7C1F7C1F7C1F781F781F7C2E
:104020001F7C3F3C7F3EFF1FDF0F000000000000B1
:104030000000000000000000000000000000000080
:10404000F803FC0F3E1F1E3E1F3C1F7CFF7FFF7FBF
:10405000007C007C003C003E071FFF0FFE030000B9
:104060000000000000000000FF01E103C003C007E2
:10407000C007C007FF7FFF7FC007C007C007C0079A
:10408000C007C007C007C007C007C007C007C007F8
:10409000C007000000000000000000000000000059
:1040A0000000000000000000EF07FF1F7F3E1F3CE4
:1040B0001F7C1F7C1F781F781F781F7C1F7C3F3C54
:1040C0007F3EFF1FDF0F1E001E001E007C38F83FE2
:1040D000003C003C003C003C003C003CFC3DFE3F02
:1040E0009E3F1F3F1F3E1F3C1F3C1F3C1F3C1F3C71
:1040F0001F3C1F3C1F3C1F3C1F3C000000000000F9
:1041000000000000F001F0010000000000000000CD
:10411000E07FE07FE001E001E001E001E001E0019B
:10412000E001E001E001E001E001E001E001000068
:104130000000000000000000F800F800000000008F
:1041400000000000F83FF83FF800F800F800F80021
:10415000F800F800F800F800F800F800F800F8009F
:10416000F800F800F800F000F071E07F003C003C3F
:10417000003C003C003C003C1F3C3E3C7C3CF83C8E
:10418000F03DE03DC03FC03FE03FF03DF83C7C3CAF
:104190003E3C1F3C1F3C00000000000000000000EF
:1041A000F07FF001F001F001F001F001F001F00109
:1041B000F001F001F001F001F001F001F001F00177
:1041C000F001F001F001F001F0010000000000003A
:1041D00000000000000000000000000000000000DF
:1041E0009EF7FFFFFFFFFFFFE7FBE7F9C7F1C7F10E
:1041F000C7F1C7F1C7F1C7F1C7F1C7F1C7F10000B7
:1042000000000000000000000000000000000000AE
:1042100000000000FC3DFE3F9E3F1F3F1F3E1F3C35
:104220001F3C1F3C1F3C1F3C1F3C1F3C1F3C1F3CB6
:104230001F3C000000000000000000000000000023
:104240000000000000000000F007FC1F3E3E1F3C85
:104250001F7C0F780F780F780F780F781F7C1F3C2A
:104260003E3EFC1FF00700000000000000000000C0
:10427000000000000000000000000000F83DFE3FCC
:104280003E3F1F3E0F3C0F3C0F3C0F3C0F3C0F3C92
:104290001F3C1E3E3E3FFC3FF83F003C003C003CC4
:1042A000003C003C00000000000000000000000096
:1042B000EE07FE1F7E3E1E3C1E7C1E781E781E787A
:1042C0001E781E781E7C3E7C7E3EFE1FDE0F1E008A
:1042D0001E001E001E001E00000000000000000066
:1042E000000000007F1FFF1FE71FC71F871F001F61
:1042F000001F001F001F001F001F001F001F001FC6
:10430000001F00000000000000000000000000008E
:104310000000000000000000FC07FE1F0E1E003E13
:10432000003E003FE01FFC07FE003E001E001E0096
:104330003E3CFC3FF01F00000000000000000000B9
:10434000000000000000800780078007FF7FFF7FDC
:104350008007800780078007800780078007800725
:1043600080078007C007FF03FF0100000000000076
:10437000000000000000000000000000000000003D
:104380001E3C1E3C1E3C1E3C1E3C1E3C1E3C1E3C5D
:104390001E3C1E3C3E3C7E3CFE3EFE1FDE0F0000EF
:1043A000000000000000000000000000000000000D
:1043B0000000000007F00F780F781E3C1E3C1E3EE8
:1043C0003C1E3C1E780F780FF00FF007F007E0035B
:1043D000E0030000000000000000000000000000FA
:1043E000000000000000000003F0E3F1E3F3E7F356
:1043F000F7F3F7F3F77F777F7F7F7F7F7F7F3E3E07
:104400003E3E3E3E3E3E0000000000000000000038
:104410000000000000000000000000000F7C1E3EB5
:104420003C3E3C1FF80FF007F007E003F007F807E9
:10443000F80F7C1E3E3E1F3C1F780000000000006D
:10444000000000000000000000000000000000006C
:1044500007F80F780F7C1E3C1E3C3C1E3C1E3C1F88
:10446000780FF80FF007F007E003E003C003C00384
:10447000C0038007800F007F0000000000000000E4
:1044800000000000FF3FFF3F1F003E007C00F800DF
:10449000F001E003C007800F001F001E003CFF7FFB
:1044A000FF7F00000000000000000000FE01E003AC
:1044B000C003C003C003C003E001E001E001C0018C
:1044C000C003803F803FC003C001E001E001E00184
:1044D000C003C003C003C003E003FE017E00000070
:1044E000C001C001C001C001C001C001C001C001C4
:1044F000C001C001C001C001C001C001C001C001B4
:10450000C001C001C001C001C001C001C001C001A3
:10451000C0010000C03FE003E001E001E001E00174
:10452000C001C003C003C001E001FE00FE00E001C5
:10453000C001C003C003C001E001E001E001E001EF
:10454000E003C03F003F000000000000000000004A
:104550000000000000000000000000000000073F15
:10456000C77FE773FFF17EF000000000000000004D
:10457000000000000000000000000000000000003B
:10458000000000000000000000000000000000002B
:10459000000000000000000000000000000000001B
:1045A0000000000C000C000C000C000C000C000CB7
:1045B000000C000C000C000C0000000C000C0000B3
:1045C000000000000000001B001B001B001B001B64
:1045D00000000000000000000000000000000000DB
:1045E0000000000000000000000080198019801900
:1045F0008019C07FC07F80190033C07FC07F003327
:104600000033003300330000000000000000001EF3
:10461000003F807580650074003C001E0007800527
:10462000806580658075003F001E00040004000066
:104630000000007000D840D8C0D880D900730006B0
:10464000000C801BC036C066C046C0068003000058
:10465000000000000000001E003F00330033003364
:10466000001E000CC03CC066806380618063C03E59
:10467000801C0000000000000000000C000C000C7A
:10468000000C000C00000000000000000000000012
:104690000000000000000000000000008000000199
:1046A0000003000600060004000C000C000C000CC7
:1046B000000C000C0004000600060003000180004E
:1046C000002000100018000C000C0004000600067A
:1046D00000060006000600060004000C000C00188E
:1046E000001000200000000C002D003F001E0033D1
:1046F00000000000000000000000000000000000BA
:104700000000000000000000000000000000000C9D
:10471000000C000C000CC0FFC0FF000C000C000CD3
:10472000000C00000000000000000000000000007D
:104730000000000000000000000000000000000079
:10474000000000000000000C000C00040004000841
:104750000000000000000000000000000000000059
:104760000000001E001E000000000000000000000D
:104770000000000000000000000000000000000039
:104780000000000000000000000000000000000C1D
:10479000000C000000000000000000030003000304
:1047A0000006000600060006000C000C000C000CC1
:1047B0000018001800180000000000000000001E93
:1047C000003F0033806180618061806D806D806119
:1047D000806180610033003F001E00000000000087
:1047E00000000006000E001E00360026000600062F
:1047F000000600060006000600060006000600008F
:10480000000000000000001E003F80738061806196
:10481000800100030006000C001800300060807F5B
:10482000807F0000000000000000001C003E0063CC
:1048300000630003000E000E000380018001806110
:104840008073003F001E0000000000000000000612
:10485000000E000E001E001E001600360036006618
:10486000807F807F00060006000600000000000038
:104870000000007F007F006000600060006E007F2D
:1048800080638001800180618073003F001E000012
:10489000000000000000001E003F803380610060C7
:1048A000006E007F80738061806180618033003F93
:1048B000001E0000000000000000807F807F80015B
:1048C0000003000300060006000C000C000C0008AA
:1048D0000018001800180000000000000000001E72
:1048E000003F8063806180610021001E003F806185
:1048F000806180618061003F001E000000000000B8
:104900000000001E003F0073806180618061807341
:10491000803F801D800180610073003F001E000009
:104920000000000000000000000000000000000C7B
:10493000000C000000000000000000000000000C5F
:10494000000C00000000000000000000000000005B
:1049500000000000000C000C00000000000000003F
:104960000000000C000C000400040008000000001F
:104970000000000080008003000E00380060003856
:10498000000E800380000000000000000000000016
:1049900000000000000000000000807F807F000019
:1049A0000000807F807F0000000000000000000009
:1049B0000000000000000000000000000040007047
:1049C000001C000780010007001C00700040000070
:1049D00000000000000000000000001F803FC071C8
:1049E000C060C000C00180030007000E000C000C76
:1049F0000000000C000C0000000000000000001E81
:104A0000003F803180718063806F806D806D806F2A
:104A1000806700600032003E001C000000000000C3
:104A20000000000E000E001B001B001B001B80314D
:104A30008031803F803F8031C060C060C060000036
:104A4000000000000000007C007E00630063006343
:104A50000063007E007E0063806180618063007F70
:104A6000007E0000000000000000001E003F8031BA
:104A70008061006000600060006000600060806134
:104A80008031003F001E0000000000000000007C9C
:104A9000007F0063806380618061806180618061EC
:104AA000806100630063007E007C00000000000065
:104AB0000000807F807F0060006000600060007FF9
:104AC000007F0060006000600060807F807F0000E9
:104AD000000000000000807F807F006000600060B8
:104AE0000060007F007F0060006000600060006088
:104AF00000600000000000000000001E003F803148
:104B0000806100600060006080638063806180611C
:104B10008031803F001E0000000000000000806126
:104B200080618061806180618061807F807F806141
:104B30008061806180618061806100000000000010
:104B40000000003F003F000C000C000C000C000CAB
:104B5000000C000C000C000C000C003F003F00009B
:104B600000000000000080018001800180018001C0
:104B70008001800180018001806180618073003F3D
:104B8000001E0000000000000000C06080610063A3
:104B900000660066006C0078007C006600660063BA
:104BA00080618061C06000000000000000000060C3
:104BB00000600060006000600060006000600060F5
:104BC000006000600060807F807F000000000000C7
:104BD0000000C071C071C07BC07AC06AC06AC06E7C
:104BE000C064C060C060C060C060C060C0600000E1
:104BF00000000000000080718071807980798079E8
:104C0000806D806D806D8065806780678067806360
:104C100080630000000000000000001E003F003321
:104C2000806180618061806180618061806180617C
:104C30000033003F001E0000000000000000007E66
:104C4000007F80638061806180618063007F007E7F
:104C50000060006000600060006000000000000074
:104C60000000001E003F0033806180618061806130
:104C700080618061806580670033803F401E000056
:104C8000000000000000007E007F80638061806182
:104C90008063007F007E0066006300638061806146
:104CA000C0600000000000000000000E001F803106
:104CB000803100300038001E000780038061806171
:104CC0008031003F001E0000000000000000C0FF17
:104CD000C0FF000C000C000C000C000C000C000CC1
:104CE000000C000C000C000C000C00000000000088
:104CF000000080618061806180618061806180618D
:104D000080618061806180618073003F001E0000CF
:104D1000000000000000C060C060C06080318031D1
:104D20008031001B001B001B001B000E000E000E3C
:104D300000040000000000000000C0C0C0C0C0C0EF
:104D4000C0C0C0C0C0CC804C804C805E80528052BD
:104D50008073806180610000000000000000C0C01E
:104D6000806080610033003B001E000C000C001EC0
:104D7000001F003B80718061C0C000000000000087
:104D80000000C0C08061806100330033001E001E3F
:104D9000000C000C000C000C000C000C000C0000BF
:104DA000000000000000803F803F800100030003FE
:104DB0000006000C000C0018001800300060807F16
:104DC000807F000000000000000F000F000C000CAE
:104DD000000C000C000C000C000C000C000C000C73
:104DE000000C000C000C000C000F000F000000185D
:104DF00000180018000C000C000C000C0006000647
:104E0000000600060003000300030000000000008D
:104E1000001E001E00060006000600060006000632
:104E20000006000600060006000600060006000652
:104E3000001E001E0000000C000C001E00120033BB
:104E4000003380618061000000000000000000006D
:104E50000000000000000000000000000000000052
:104E60000000000000000000000000000000000042
:104E70000000000000000000E0FF0000000000381B
:104E80000018000C000000000000000000000000FE
:104E90000000000000000000000000000000000012
:104EA00000000000000000000000001F803F806143
:104EB0008001801F803F80618063807FC038000058
:104EC0000000000000000060006000600060006EF4
:104ED000007F807380618061806180618073007F6A
:104EE000006E000000000000000000000000000054
:104EF0000000001E003F80738061006000608061E0
:104F00008073003F001E00000000000000008001D0
:104F1000800180018001801D803F807380618061FD
:104F2000806180618073803F801D00000000000070
:104F300000000000000000000000001E003F0073A1
:104F40008061807F807F00608071003F001E0000D4
:104F5000000000000000C007C00F000C000C807FA4
:104F6000807F000C000C000C000C000C000C000CEE
:104F7000000C000000000000000000000000000025
:104F8000801D803F8073806180618061806180735B
:104F9000803F801D80018063007F003E0000006034
:104FA000006000600060006F807F807180618061C0
:104FB000806180618061806180610000000000008C
:104FC00000000006000600000000003E003E000653
:104FD00000060006000600060006000600060000A7
:104FE000000000000006000600000000003E003E39
:104FF0000006000600060006000600060006000681
:1050000000060046007E003C00000060006000607A
:105010000060806100630066006C007C00760063C5
:1050200000638061C0600000000000000000003EDE
:10503000003E000600060006000600060006000608
:105040000006000600060006000600000000000042
:105050000000000000000000000080DDC0FFC0CEA6
:10506000C0CCC0CCC0CCC0CCC0CCC0CCC0CC00006C
:105070000000000000000000000000000000006FC1
:10508000807F8071806180618061806180618061EA
:10509000806100000000000000000000000000002F
:1050A0000000001E003F807380618061806180612C
:1050B0008073003F001E00000000000000000000A0
:1050C00000000000006E007F80738061806180615D
:1050D00080618073007F006E00600060006000608F
:1050E0000000000000000000801D803F8073806190
:1050F0008061806180618073803F801D80018001BC
:105100008001800100000000000000000000006736
:10511000803F003900300030003000300030003077
:10512000003000000000000000000000000000004F
:105130000000001E803F80610060007F803F800192
:105140008061007F001E00000000000000000000E1
:10515000000800180018007F007F001800180018D1
:10516000001800180018801F800F000000000000C9
:10517000000000000000000000008061806180618C
:1051800080618061806180618063807F803D0000FC
:105190000000000000000000000000000000C060EF
:1051A000803180318031001B001B001B000E000E7F
:1051B00000060000000000000000000000000000E9
:1051C000000080DD80DD80DD005500550055007752
:1051D0000077002200220000000000000000000014
:1051E000000000000000806100330033001E000C4E
:1051F000000C001E0033003380610000000000003E
:1052000000000000000000008061806180310033F8
:105210000033001B001B001B000E000E000E001CC4
:10522000007C007000000000000000000000C07F53
:10523000C07F800100030006000C00180030C07F12
:10524000C07F000000000000800380070006000609
:10525000000600060006000E001C001C000E0006E2
:105260000006000600060006800780030006000610
:1052700000060006000600060006000600060006FE
:1052800000060006000600060006000600060006EE
:105290000038003C000C000C000C000C000C000E50
:1052A00000070007000E000C000C000C000C000CA6
:1052B000003C00380000000000000000000000007A
:1052C00000008038807F00470000000000000000E0
:1052D00000000000000000000000000000000000CE
:1052E000000000000000000000000000001000109E
:1052F000001000100010001000000010000000005E
:105300000028002800280000000000000000000025
:105310000000000000240024007C00240048007CE1
:1053200000480048000000000038005400500038D9
:1053300000140054005400380010000000200054F5
:10534000005800300028005400140008000000003D
:1053500000100028002800100034004800480034E5
:10536000000000000010001000100000000000000D
:1053700000000000000000000008001000200020D5
:105380000020002000200020001000080020001055
:1053900000080008000800080008000800100020AD
:1053A000001000380010002800000000000000007D
:1053B000000000000000000000100010007C001041
:1053C00000100000000000000000000000000000CD
:1053D000000000000000001000100010000000009D
:1053E0000000000000000038000000000000000085
:1053F000000000000000000000000000000000109D
:10540000000000000008000800100010001000104C
:105410000020002000000000003800440044005438
:105420000044004400440038000000000010003038
:1054300000500010001000100010001000000000CC
:105440000038004400440004000800100020007CE4
:1054500000000000003800440004001800040004AC
:105460000044003800000000000800180028002850
:105470000048007C0008000800000000007C00409C
:1054800000400078000400040044003800000000E0
:1054900000380044004000780044004400440038D4
:1054A00000000000007C0004000800100010002034
:1054B00000200020000000000038004400440038B4
:1054C000004400440044003800000000003800445C
:1054D00000440044003C0004004400380000000088
:1054E000000000000010000000000000000000109C
:1054F000000000000000000000000010000000009C
:10550000000000100010001000000000000C00302F
:1055100000400030000C000000000000000000000F
:105520000000007C0000007C000000000000000083
:105530000000000000600018000400180060000077
:1055400000000000003800440004000800100010B3
:10555000000000100000000000380044004C00541F
:10556000005C0040004000380000000000100028EF
:10557000002800280028007C0044004400000000AF
:10558000007800440044007800440044004400785F
:10559000000000000038004400400040004000408F
:1055A000004400380000000000700048004400443F
:1055B000004400440048007000000000007C0040EF
:1055C0000040007C004000400040007C00000000E3
:1055D000007C004000400078004000400040004057
:1055E000000000000038004400400040005C00441F
:1055F0000044003800000000004400440044007CE7
:105600000044004400440044000000000038001042
:105610000010001000100010001000380000000002
:1056200000040004000400040004000400440038E6
:105630000000000000440048005000600050004896
:1056400000480044000000000040004000400040CE
:10565000004000400040007C000000000044006C5E
:10566000006C00540044004400440044000000006A
:1056700000440064006400540054004C004C00449A
:10568000000000000038004400440044004400448E
:10569000004400380000000000780044004400444A
:1056A0000078004000400040000000000038004446
:1056B000004400440044004400540038000400004A
:1056C000007800440044004400780048004800444A
:1056D00000000000003800440040003000080004D2
:1056E0000044003800000000007C00100010001092
:1056F00000100010001000100000000000440044E2
:10570000004400440044004400440038000000000D
:105710000044004400440028002800280010001025
:105720000000000000440044005400540054006C89
:105730000028002800000000004400280028001075
:10574000001000280028004400000000004400442D
:1057500000280028001000100010001000000000B9
:10576000007C000400080010001000200040007CB5
:1057700000000000001800100010001000100010C1
:105780000010001000100018002000200010001071
:105790000010001000080008000000000030001099
:1057A0000010001000100010001000100010003059
:1057B0000010002800280044000000000000000045
:1057C00000000000000000000000000000000000D9
:1057D00000000000000000FE00200010000000009B
:1057E00000000000000000000000000000000000B9
:1057F00000380044003C0044004C0034000000002D
:105800000040004000580064004400440064005818
:10581000000000000000000000380044004000408C
:105820000044003800000000000400040034004C74
:1058300000440044004C0034000000000000000060
:1058400000380044007C00400044003800000000A4
:10585000000C0010007C0010001000100010001060
:1058600000000000000000000034004C0044004430
:10587000004C0034000400780040004000580064F0
:1058800000440044004400440000000000100000F8
:105890000070001000100010001000100000000048
:1058A0000010000000700010001000100010001028
:1058B000001000E000400040004800500060005030
:1058C00000480044000000000070001000100010AC
:1058D0000010001000100010000000000000000088
:1058E000007800540054005400540054000000009C
:1058F00000000000005800640044004400440044DC
:105900000000000000000000003800440044004493
:10591000004400380000000000000000005800644F
:1059200000440044006400580040004000000000B3
:105930000034004C00440044004C003400040004D7
:10594000000000000058006400400040004000409B
:105950000000000000000000003800440030000893
:1059600000440038000000000020002000780020E3
:1059700000200020002000180000000000000000AF
:105980000044004400440044004C00340000000087
:1059900000000000004400440028002800280010F7
:1059A0000000000000000000005400540054006C8F
:1059B000002800280000000000000000004400282B
:1059C000001000100028004400000000000000004B
:1059D000004400440028002800100010001000605F
:1059E00000000000007C0008001000200040007C47
:1059F000000000000018001000100010002000201F
:105A0000001000100010001800100010001000100E
:105A100000100010001000100010001000300010E6
:105A200000100010000800080010001000100030E6
:105A30000000000000000074004C000000000000A6
:105A4000000000000000000000000000010203044C
:105A50000607080900000000010203044572726F86
:105A60007220777269746520706F6C6172697479E5
:105A70000A0000004572726F7220777269746520A7
:105A80006F75747075740A004572726F7220777248
:105A900069746520696E69740A0000004572726F4E
:105AA0007220777269746520636F6E6669670A0099
:105AB00052656164206572726F720A002B000000EB
:105AC0002D0000002A0000003120322033000000A9
:105AD00034203520360000003720382039000000FF
:105AE0002A20302023000000256C64002A3A6F70C1
:105AF00020233A636C720000256C6420257300003B
:105B00002A3A63686720233A3D0000003D256C6413
:105B1000000000002A3A75736520233A7270740001
:105B2000232D302B2000686C4C0065666745464786
:105B30000030313233343536373839414243444509
:105B40004600303132333435363738396162636478
:045B50006566000086
:085B54007CA6FF7F01000000A8
:045B5C00B501000887
:045B600091010008A7
:105B64000100000010000000101A0000303200088C
:105B74000B1200007C450008070A0000D8520008F8
:105B84000024F4002800002000000000700500201C
:105B9400D80500204006002000000000000000009E
:105BA40000000000000000000000000000000000F1
:105BB40000000000000000000000000000000000E1
:105BC40000000000000000000000000000000000D1
:045BD40000000000CD
:040000050800288542
:00000001FF
